:020000040000FA
:1000000085018316803081009501D83085009901E3
:1000100058309F00FF2390008312073099008E0113
:100020008F01900181018B0105308500851610300C
:10003000A0003820A00B19284720A1012D2047201F
:100040005030851D5130A1002D2047205030851D96
:100050005130A1002D20382017280830A000A10D14
:10006000031C3428382035284720A00B2F280800EF
:100070000B1D3828E63081000B11053085000B1D63
:100080003F28E63081000B110630850008000B1D6B
:100090004728C93081000B11053085000D309F00C5
:1000A0000630A200A20B52289F149F185528193021
:1000B00003101E02031872280B1D5C28C930810032
:1000C0000B11063085000D309F000630A200A20BF8
:1000D00067289F149F186A28193003101E020318FE
:1000E00072280800851200308500353090000A30F3
:1000F000A2008E018F010C100C1C7C28A20B792809
:0C0100008E018F0190013430851608003C
:02400E00C43FAD
:10421000470065006E0065007200610074002E00AA
:1042200066007200650069006E006100670065004D
:10423000310035002F00300036002F0030003900EB
:1042400076006500720073002E002000340020000C
:104250007200650067006C006100670065003A004D
:0E42600031002C0035004100200035007300B5
:00000001FF
